:0600000000F067EF00F0C4
:10000800FACF02F0FBCF03F0E9CF04F0EACF05F016
:10001800E1CF06F0E2CF07F0D9CF08F0DACF09F048
:10002800F3CF0AF0F4CF0BF0F6CF0CF0F7CF0DF0CA
:10003800F8CF0EF0F5CF0FF09EA423D09E94B1A078
:1000480014D0B190B2CF5AF05B6AB3CF58F0596A66
:100058006CC056F06DC057F0A1A202D0564A572A7C
:10006800016E010E6B6E01500CD0A192000EB36EA2
:10007800000EB26E000E6D6E000E6C6E00F000F099
:10008800B180A1A203D0A1926C4A6D2A0FC0F5FFDE
:100098000EC0F8FF0DC0F7FF0CC0F6FF0BC0F4FF51
:1000A8000AC0F3FF09C0DAFF08C0D9FF07C0E2FFA2
:1000B80006C0E1FF05C0EAFF04C0E9FF03C0FBFF7B
:0A00C80002C0FAFF11003AEF06F043
:100100000001000A006400E8031027202533642C56
:1001100025303364002E253033646B487A000000AC
:10012000000EC16EF00E926ECF0E936ECD8ECD8A04
:10013000CD88CD96CD84CD92CD909E909D90A2827B
:10014000B18EB19AB198B184B196B182B190A192B9
:10015000A0829F84BD86BD94BD82BD80500EBE6EC0
:10016000C30EBF6E9E949D8472EC05F0DDEC06F02C
:10017000D08EF28EF28CCD8080BA0FD0000E646EDD
:10018000000E656E000E666E000E676E000E696EE4
:10019000010E686E366E000E0ED0A80E646E0E0E46
:1001A000656EF90E666EFF0E676E000E696E640E68
:1001B000686E366E010E6A6E36506FEC03F020EEFC
:1001C00068F0DECF10F0DDCF11F0000E11BEFF0E93
:1001D000126E136E60C014F061C015F062C016F0AC
:1001E00063C017F0CFEC05F010C052F011C053F00F
:1001F00012C054F013C055F055BE0ED05550800AB1
:10020000450F08E19A0E545C05E1CA0E535C02E109
:10021000000E525CD8A040D0366E200E496E36508B
:10022000366E200E4A6E3650366E4F0E4B6E36507E
:10023000366E750E4C6E3650366E740E4D6E3650F0
:10024000366E200E4E6E3650366E6F0E4F6E365036
:10025000366E660E506E3650366E200E3E6E36503E
:10026000366E520E3F6E3650366E610E406E365010
:10027000366E6E0E416E3650366E670E426E3650DA
:10028000366E650E436E3650366E200E446E365016
:10029000366E200E456EB3D052C01BF053C01CF01A
:1002A00054C01DF055C01EF0400E1F6E420E206E51
:1002B0000F0E216E000E226E22EC04F01BC036F0F1
:1002C0001CC037F01DC038F01EC039F036C047F0F2
:1002D00037C048F0400E146E420E156E0F0E166EAB
:1002E000000E176E52C010F053C011F054C012F03F
:1002F00055C013F0A6EC04F010C01BF011C01CF0A8
:1003000012C01DF013C01EF0E80E1F6E030E206E0B
:10031000000E216E000E226E22EC04F01BC036F09F
:100320001CC037F01DC038F01EC039F036C03AF09E
:1003300037C03BF052C010F053C011F054C012F05F
:1003400055C013F0E80E146E030E156E000E166EF7
:10035000000E176EA6EC04F010C036F011C037F096
:1003600012C038F013C039F036C03CF037C03DF051
:10037000000E1F6E490E1E6E010E216E0B0E206EBA
:1003800047C022F048C023F03AC024F03BC025F01B
:1003900019EC02F0000E1F6E3E0E1E6E010E216E55
:1003A000150E206E3CC022F03DC023F019EC02F087
:1003B00048504710D8A418D0366E200E4C6E3650D8
:1003C000366E200E4D6E36504E50300AD8A40CD0EA
:1003D000366E200E4E6E36504F50300AD8A404D0E0
:1003E000366E200E4F6E365068046910D8B408D0AF
:1003F000366E200E406E3650366E200E416E3650F0
:10040000000EE7EC06F0000E166E490E156E66EC57
:1004100006F0400EE7EC06F0000E166E3E0E156E6E
:1004200066EC06F0000E116EC80E106E9EEC06F023
:10043000A3D6000E2B6E220E2A6E3FD13550250A10
:10044000D8B409D01EC0D9FF1FC0DAFF35C0DFFF06
:100450001E4A1F2A32D1000E346E000E336E266EF5
:10046000000E326E265003D03284204A212A20C04A
:10047000F6FF21C0F7FF0800F550300AD8B4F4D7D2
:1004800020C0F6FF21C0F7FF0800F55051EC06F040
:10049000D8A032D0000E346E000E336E33C010F090
:1004A00034C011F0000E136E0A0E126E1DEC06F031
:1004B00010C033F011C034F0D00E266EFF0E276E40
:1004C00020C0F6FF21C0F7FF0800F550286E296A0A
:1004D00026502826275029222850332629503422F6
:1004E000204A212A20C0F6FF21C0F7FF0800F5505E
:1004F00051EC06F0D8B0D2D720C0F6FF21C0F7FFEC
:10050000204A212A0800F5CF35F03550000AD8B42A
:10051000DFD0640AD8B403D00D0AD8A4CED02AC044
:10052000D9FF2BC0DAFFDECF2DF0DDCF2EF0020E8B
:100530002A26000E2B222E50800AF36E800EF35CCA
:10054000000ED8B42D5CD8B006D0030E32122D6C3C
:100550002E1ED8B02E2A266E010E356E265035502E
:10056000050AD8B416D03550020D010EF324F66EEC
:10057000010EF420F76E0900F5CF26F00900F5CF43
:1005800027F026502D5C27502E58D8A002D0352AAF
:10059000E6D734503310D8B409D032C026F0030E59
:1005A0002616D8B403D03306D8A03406800E35BE44
:1005B0007F0E266E3350355C3450800A2658D8B0F2
:1005C00007D03550335E000E35BEFF0E345A04D0CE
:1005D000000E346E000E336E32A41ED032C026F0F0
:1005E000030E2616D8B408D01EC0D9FF1FC0DAFFEC
:1005F0002D0EDF6E1E4A1F2A34503310D8B42DD072
:100600001EC0D9FF1FC0DAFF300EDF6E1E4A1F2A40
:100610003306D8A03406F0D734503310D8B40FD0F6
:100620001EC0D9FF1FC0DAFF200EDF6E1E4A1F2A30
:100630003306D8A0340634503310D8A4F1D732C0D2
:1006400026F0030E2616D8B408D01EC0D9FF1FC04E
:10065000DAFF2D0EDF6E1E4A1F2A35C02CF029D07E
:100660002C50020D010EF324F66E010EF420F76EED
:100670000900F5CF12F00A00F5CF13F02DC010F0ED
:100680002EC011F0A4EC05F010C018F011C019F044
:10069000000E1B6E0A0E1A6EFAEC05F01850300FA1
:1006A000356E1EC0D9FF1FC0DAFF35C0DFFF1E4AFE
:1006B0001F2A2C062C28D8A4D3D720C0F6FF21C08F
:1006C000F7FF204A212A0800F5CF35F03566B6D667
:1006D0001EC0D9FF1FC0DAFF000EDF6E1200585097
:1006E0002B6E2A6A56502C6E57502D6E2E6A2F6A2A
:1006F0002DC02FF02CC02EF02D6A2C6A2A502C24ED
:10070000306E2B502D20316E000E2E20326E000EDA
:100710002F20336E5A503024106E5B503120116EF2
:10072000000E3220126E000E3320136E0A0E146E6D
:10073000000E156E000E166E000E176ECFEC05F053
:1007400010C05CF011C05DF012C05EF013C05FF02D
:1007500064505C241B6E65505D201C6E66505E20EC
:100760001D6E67505F201E6E20EE68F0DECF1FF01A
:10077000DDCF20F0000E20BEFF0E216E226E22EC97
:1007800004F01BC060F01CC061F01DC062F01EC010
:1007900063F06A50D8B455D020EE68F0DE52DD50D8
:1007A000800A800F020ED8B4DF5CD8A04AD068C09F
:1007B00010F069C011F0000E136E020E126E1AECEA
:1007C00005F010C02AF011C02BF0000E2BBEFF0E5A
:1007D0002C6E2D6E64505C24106E65505D20116E81
:1007E00066505E20126E67505F20136E20EE68F038
:1007F000DECF14F0DDCF15F0000E15BEFF0E166E25
:10080000176EA6EC04F010C02EF011C02FF012C02D
:1008100030F013C031F03150800A326E2A502E5C15
:100820002B502F582C5030582D50800A3258D8A0B9
:1008300008D0010E6026000E6122000E6222000E1A
:1008400063221200236E000E256E23502250800A70
:10085000800F08E1000E215C05E1000E205C02E142
:10086000000E1F5CD8B00CD0221E211E201E1F6C53
:10087000000E202221222222236E010E256E2350FB
:100880001E50800A800F08E1000E1D5C05E1000E7D
:100890001C5C02E1000E1B5CD8B00AD01E1E1D1E9F
:1008A0001C1E1B6C000E1C221D221E22010E251A6E
:1008B000000E266E000E276E000E286E000E296EAA
:1008C00022501F1020102110D8B42CD0236E010EFE
:1008D000246E235006D0D8901F362036213622367B
:1008E000242A22AEF8D7D89026362736283629363D
:1008F0001F501B5C20501C5821501D5822501E5860
:10090000D8A009D01F501B5E20501C5A21501D5AE0
:1009100022501E5A2680D8902232213220321F3295
:10092000242EE1D72550D8B408D0291E281E271E12
:10093000266C000E27222822292226C01BF027C061
:100940001CF028C01DF029C01EF01200186E000E09
:100950001A6E18501350800A800F08E1000E125CC6
:1009600005E1000E115C02E1000E105CD8B00CD065
:10097000131E121E111E106C000E112212221322C1
:10098000186E010E1A6E18501750800A800F08E179
:10099000000E165C05E1000E155C02E1000E145C11
:1009A000D8B008D0171E161E151E146C000E152286
:1009B000162217221750141015101610D8B426D06E
:1009C000186E010E196E185006D0D89014361536D0
:1009D00016361736192A17AEF8D71450105C155072
:1009E00011581650125817501358D8A008D0145048
:1009F000105E1550115A1650125A1750135AD890AB
:100A00001732163215321432192EE7D71A50D8B4CD
:100A100008D0131E121E111E106C000E112212227D
:100A2000132210C010F011C011F012C012F013C048
:100A300013F01200146E000E166E14501350800A3C
:100A4000F36E800EF35C000ED8B4125CD8B008D000
:100A5000126C131ED8B0132A146E010E166E1450A9
:100A60001150800AF36E800EF35C000ED8B4105C57
:100A7000D8B006D0106C111ED8B0112A010E161A6B
:100A8000000E186E000E176E13501210D8B41ED040
:100A9000146E010E156E145004D0D8901236133611
:100AA000152A13AEFAD7D890173618361250105CA4
:100AB00013501158D8A005D01250105E1350115A7F
:100AC0001780D89013321232152EEDD71650D8B4A5
:100AD00004D0176C181ED8B0182A17C010F018C010
:100AE00011F012008A98000E116E280E106E8CEC18
:100AF00006F0030EAFEC06F0000E116E050E106E40
:100B00008CEC06F08A8A8A9A850EE82EFED700F0D1
:100B10008A8A8A9A000E116E050E106E8CEC06F011
:100B2000020EAFEC06F0850EE82EFED700F0280E80
:100B3000D2EC06F0080ED2EC06F00C0ED2EC06F069
:100B4000060ED2EC06F01200000E166E000E156EA8
:100B500013501210D8B41ED0146E010E176E14501C
:100B600004D0D89012361336172A13AEFAD7D8907D
:100B7000153616361250105C13501158D8A005D0F7
:100B80001250105E1350115A1580D8901332123241
:100B9000172EEDD715C010F016C011F01200000E80
:100BA000186E000E196E000E1A6E000E1B6E10A04D
:100BB00008D0145018261550192216501A22175012
:100BC0001B22D8901436153616361736D8901332A5
:100BD0001232113210321350101011101210D8A40A
:100BE000E6D718C010F019C011F01AC012F01BC0DF
:100BF00013F012001B501A10D8B41AD01C6E010E3C
:100C00001D6E1C5004D0D8901A361B361D2A1BAE00
:100C1000FAD71A50185C1B501958D8A004D01A5093
:100C2000185E1B50195AD8901B321A321D2EF1D75C
:100C300018C018F019C019F0120010501202F3CFAA
:100C400014F0F4CF15F010501302F3CFF4FFF36A51
:100C5000F3501426F450152211501202F3CFF4FF72
:100C6000F36AF3501426F450152214C010F015C086
:100C700011F012006D6A6C6A780EF66E0D0EF76E4A
:100C8000000EF86E00EE56F010EE16F00900F5CFEB
:100C9000EEFFE550E150FAE1000EF86E000190EF32
:100CA00000F0E8CF12F0106E000E116E10503A0EE8
:100CB000125CD8B007D02F0E126404D0106E010E53
:100CC000116E105011C010F0103012008A8809D037
:100CD00015C0D9FF16C0DAFFDF50C7EC06F0154A81
:100CE000162A15C0D9FF16C0DAFFDF50D8B412009B
:100CF000EFD7E8CF13F013C012F0123A0F0E12160E
:100D00000F0E12168950F00B1210896E8A8A8A9A79
:100D10001350AFEC06F0120008D0060E126E300E23
:100D2000E82EFED7122EFCD700D01006D8A0110650
:100D30001028D8B41128D8B41200EFD711501010D1
:100D4000D8B40CD0060E126E300EE82EFED7122E3E
:100D5000FCD700D01006D8A01106F0D71200E8CFBB
:100D600011F011C010F00F0E10168950F00B10107A
:100D7000896E8A8A8A9A1200000000000000000032
:100D8000000000000000A80EF9FF64000100E8CF99
:100D900014F08A88145079EC06F0350EE82EFED750
:100DA00000F01200E8CF14F08A98145079EC06F0A5
:100DB000350EE82EFED700F01200010ED2EC06F040
:100DC000000E116E020E106E8CEC06F01200E8CFD1
:0C0DD00015F01550800FD2EC06F0120058
:020000040020DA
:08000000FFFFFFFFFFFFFFFF00
:020000040030CA
:0E000000FF020D1EFF0080FF03C003E003405F
:00000001FF
